:1000000030050020E51100005B23000075100000A2
:1000100075100000751000007510000075100000CC
:10002000751000007510000075100000D90C00005C
:100030007510000075100000810C000043230000C3
:10004000A5110000A5110000A5110000A5110000D8
:10005000A5110000A5110000A5110000A5110000C8
:10006000A5110000A5110000A5110000A5110000B8
:10007000A5110000A5110000A5110000A5110000A8
:10008000A5110000A5110000A5110000A511000098
:10009000A5110000A5110000A5110000A511000088
:1000A000A5110000A5110000A5110000A511000078
:1000B000A5110000A5110000A5110000A511000068
:1000C000A5110000A5110000A5110000A511000058
:1000D000A5110000A5110000A5110000A511000048
:1000E000A5110000A5110000A5110000A511000038
:1000F000A5110000A5110000A5110000A511000028
:100100007BB972B90029BEBF00204FF0004106E064
:1001100008BF00281CBF6FF000414FF0FF3000F017
:10012000A5B9ADF1080C6DE904CE002909DB002B5F
:100130001ADB00F035F8DDF804E0DDE9022304B055
:100140007047404261EB4101002B1BDB00F028F8B7
:10015000DDF804E0DDE9022304B0404261EB410137
:10016000524263EB43037047524263EB430300F098
:1001700017F8DDF804E0DDE9022304B0404261EB4A
:1001800041017047524263EB430300F009F8DDF888
:1001900004E0DDE9022304B0524263EB43037047FD
:1001A0002DE9F047089E04468846002B4BD18A4231
:1001B000154667D9B2FA82F24AB1C2F1200701FAB4
:1001C00002F320FA07F7954047EA030894404FEA04
:1001D000154E230CB8FBFEF71FFA85FC0EFB1788A3
:1001E00043EA084307FB0CF1994209D9EB1807F1E0
:1001F000FF3080F01B81994240F21881023F2B446E
:100200005B1AA4B2B3FBFEF00EFB103344EA0344C6
:1002100000FB0CFCA44509D92C1900F1FF3380F038
:100220000781A44540F2048102382C4440EA07408B
:10023000A4EB0C0400271EB1D4400023C6E9004300
:100240003946BDE8F0878B4209D9002E00F0EB80DB
:100250000027C6E9000138463946BDE8F087B3FA01
:1002600083F7002F47D18B4202D3824200F2FA80FB
:10027000841A61EB030301209846002EE0D0C6E902
:100280000048DDE702B9FFDEB2FA82F2002A40F050
:100290008F80491B4FEA154E1FFA85F80127B1FBE5
:1002A000FEFC230C0EFB1C1143EA014308FB0CF17E
:1002B000994207D9EB180CF1FF3002D2994200F2B3
:1002C000CD808446591AA3B2B1FBFEF00EFB101488
:1002D00043EA044408FB00F8A04507D92C1900F1B3
:1002E000FF3302D2A04500F2B6801846A4EB080402
:1002F00040EA0C409FE7C7F1200CBB4022FA0CFEFD
:100300004EEA030E01FA07F420FA0CF521FA0CF379
:100310004FEA1E482543B3FBF8F92C0C08FB1933B0
:100320001FFA8EFA44EA034309FB0AF49C4202FADC
:1003300007F200FA07F10BD91EEB030309F1FF30B6
:1003400080F087809C4240F28480A9F102097344C6
:100350001B1BADB2B3FBF8F008FB103345EA0344B6
:1003600000FB0AFAA24508D91EEB040400F1FF3392
:100370006BD2A24569D90238744440EA0940A0FB17
:100380000289A4EB0A044C45C2464B4654D351D0D3
:10039000002E69D0B1EB0A0564EB030404FA0CFCEF
:1003A000FD40FC404CEA0505C6E90054002747E73C
:1003B000C2F1200320FA03F7954001FA02F021FA76
:1003C00003F34FEA154E3843010CB3FBFEF71FFA57
:1003D00085F80EFB173341EA034107FB08F38B4214
:1003E00004FA02F407D9691807F1FF3C2FD28B42B7
:1003F0002DD9023F2944CB1A81B2B3FBFEF00EFB8C
:10040000103341EA034100FB08F38B4207D9691816
:1004100000F1FF3C17D28B4215D902382944C91A82
:1004200040EA07473BE73746304609E70746E7E635
:100430001846FBE64145ABD2B8EB020A69EB0E0267
:1004400001381346A4E76046E9E7184695E7674692
:10045000D1E781467CE702382C4447E7ACF1020C37
:100460002B442FE7384608E73746E9E6704700BFD8
:100470000149024801F04CBFBC280000CE28000012
:100480000B6801330B60014B1B681847700E00208E
:100490002DE9F04F85B09B460E9CDFF890A0012C13
:1004A000B8BF0124012B0CBF302320231546804602
:1004B00089460194029301260A2700220AF10104C9
:1004C0000AB9AA451FD2B5FBF4F049463030C047FF
:1004D00001360122013F012FB5FBF4F14FF00A0371
:1004E00004FB1155BAFBF3FAE8D1494605F1300097
:1004F000C047BBF1030F03D1019B9C1B002C0FDCF9
:1005000005B0BDE8F08F019BBB42E3DBBBF1020FFE
:10051000E0D84946029803920136C047039AD9E7CA
:1005200049462020C047013CE8E700BFFFC99A3B8D
:10053000014B1860704700BF700E002013B502AC6D
:10054000002344F8043D02460B460348214601F0CF
:1005500083FD02B010BD00BF8104000010B54FF054
:100560002003EFF3118483F31188BFF36F8F00F042
:1005700027F8094A0123C2F840354FF08042C2F8FB
:100580007835064B4FF0FF329A62DA6284F31188B5
:10059000BFF36F8F002010BD00E0014000ED00E0D0
:1005A000054B1B68082B01BF044B1868B0FA80F09C
:1005B000400918BF002070473001001034010010BE
:1005C00008B54FF080430022C3F80C21C3F8102176
:1005D000C3F838254FF0805203F54043D2F8041495
:1005E000C3F82015D2F80814C3F82415D2F80C1457
:1005F000C3F82815D2F81014C3F82C15D2F8141427
:10060000C3F83015D2F81814C3F83415D2F81C14F6
:10061000C3F84015D2F82014C3F84415D2F82414B6
:10062000C3F84815D2F82814C3F84C15D2F82C1486
:10063000C3F85015D2F83014C3F85415D2F8341456
:10064000C3F86015D2F83814C3F86415D2F83C1416
:10065000C3F86815D2F84014C3F86C15D2F84424D6
:10066000C3F87025FFF79CFF10B1334B334A1A6073
:10067000FFF796FF18B1324BFB22C3F81825FFF79E
:100680008FFF48B12F49304B0A681B6822F00F02D8
:1006900003F00F0313430B60FFF782FF18B12B4BDE
:1006A0004FF400721A604FF08043D3F80024D20751
:1006B00044BF6FF00102C3F800244FF01023D3F8B9
:1006C0000022002A03DBD3F80432002B2FDA204B60
:1006D0000122C3F80425D3F80024002AFBD04FF0F0
:1006E00010221221C2F80012D3F80024002AFBD0F5
:1006F0004FF010231222C3F80422154B1A46D3F8E8
:1007000000140029FBD00021C3F80415D2F80034EE
:10071000002BFBD0BFF34F8F0E490F4BCA6802F47A
:10072000E0621343CB60BFF34F8F00BFFDE70B4B7D
:100730000B4A1A6008BD00BF8C5600404881030078
:1007400000F00040E40E00405802001040960240C5
:1007500000E0014000ED00E00400FA05740E002006
:100760000090D0030A2838B50446074D04D1286804
:1007700043680D215B68984728684368E1B25B686D
:100780009847204638BD00BF0800002010B5044C33
:10079000204600F023FE2046BDE81040FFF7C8BE0B
:1007A0006507000008B5044800F07AFF034B1860A5
:1007B000FFF7ECFF002008BDEE2800000800002035
:1007C00010B54FF02003EFF3118283F31188BFF3CC
:1007D0006F8F154C237833B982F31188BFF36F8F75
:1007E0006FF0440010BD013BDBB2237033B182F3E4
:1007F0001188BFF36F8F6FF00F00F3E70B4B187882
:10080000012138B1217082F31188BFF36F8F6FF02F
:100810000A00E7E7197082F31188BFF36F8F044A6B
:1008200011601870DEE700BF2A01002029010020B6
:1008300004000040F8B54FF02002EFF3118382F37B
:100840001188BFF36F8F294A1078441C147080B14F
:1008500083F31188BFF36F8F4FF08043D3F80C34CC
:1008600003F00113B3F1011F0CBF00206FF0430030
:1008700009E01F4D2F783FB1107083F31188BFF34B
:100880006F8F6FF00A00F8BD01262E7083F3118878
:10089000BFF36F8F4FF0804419B3384600F088FBE8
:1008A000C4F80071D4F80433C4F804632660D4F8A3
:1008B000002192B10022C4F800210E4A13F0010F6A
:1008C0004FF0010308BFC4F808330020C2F880319C
:1008D00000F05EFB00232B70BEE720BF40BF20BFAF
:1008E000E5E7C4F800112660F4E700BF2A01002004
:1008F0002901002000E100E070B54FF02002EFF385
:10090000118382F31188BFF36F8F244D2A789AB137
:1009100083F31188BFF36F8F4FF08042D2F81C34FD
:10092000D2F8182403F0030343F48033934314BF35
:100930006FF04300002070BD01242C7083F31188F8
:10094000BFF36F8F4FF08043154EC3F8042102258B
:10095000C3F81815C3F8045311F0030134604FF0C5
:100960001806C3F80863C3F80C21C3F81021D3D1CB
:100970001022C3F83825C3F80463D3F81824D2032F
:1009800002D4C3F80453C7E7C3F80443FFF752FF88
:100990000028C1D1034BC3F80041BDE72801002066
:1009A0000800004000E100E0F8B54FF08043054644
:1009B000D3F808C1D3F80423D3F80071D3F80403A3
:1009C000D3F80461D3F80C11D3F81041003402F0CD
:1009D000010218BF0124BCF1000F03D04FF0000C3E
:1009E000C3F808C1002F41D04FF080430027C3F85F
:1009F000007152B14FF08043224F01224FF0020CA0
:100A0000C3F80823C7F800C01A61EEB959B11D4BED
:100A10004FF08046002119602846C6F80C11FFF7F8
:100A2000CFFE0123736174B14FF080430021012494
:100A3000C3F810112846C3F80443FFF7FBFE10B9B2
:100A4000114BC3F80041F8BD4FF080430022C3F8BA
:100A500004218207DAD50222C3F80823D3F81C3414
:100A60009B07D3D10029DFD00124D0E7002ACCD0C6
:100A70004FF08043D3F80C3403F00113B3F1011F9E
:100A8000C3D1B7E7340C004000E100E0104B002276
:100A900010B4C3F840214FF02002EFF3118482F329
:100AA0001188BFF36F8F0B4AD3F80405116840F229
:100AB0004713401A20F07F40B0FBF3F003FB001314
:100AC000136084F31188BFF36F8F10BC01F0D2B9AB
:100AD000001001400C00002037B51F4800F0E0FD79
:100AE000002835D043681D4D1B680121984700241C
:100AF00040F24713C5F80845C5F840354FF4803338
:100B0000C5F84433C5F8043303F1804303F58A5331
:100B10004FF400321C601B680193019B104B0121B4
:100B2000C3F880211120224600F056FA112000F06F
:100B30002FFA0C4A012313602B60D5F8043503F219
:100B4000471323F07F43C5F84035204603B030BD3E
:100B50004FF0FF30FAE700BFF52800000010014019
:100B600000E100E0081001404CF6690270B5B0F1F8
:100B7000FF3F08BF10464FF02003EFF3118483F3CB
:100B80001188BFF36F8F1349134DD1F804352E68C8
:100B900001389042A8BF10469A1B22F07F4240F2D3
:100BA000471502F5A37220EAE07005FB0020B0FBB8
:100BB000F5F005FB0060C31A23F07F431F2B98BF9D
:100BC000401920F07F40C1F8400584F31188BFF33D
:100BD0006F8F70BD001001400C0000204FF020020C
:100BE000EFF3118382F31188BFF36F8F084AD2F8B5
:100BF0000405084A1268801A20F07F4040F247122C
:100C0000B0FBF2F083F31188BFF36F8F704700BF22
:100C1000001001400C00002004488168406A8842AE
:100C200003D003494FF080520A607047E80000206B
:100C300004ED00E0044800232021C2180133302BCA
:100C400082F80013F9D1704700E100E0094A0A492F
:100C5000936809689966094958664B6843F0805360
:100C60004B60002383F31188BFF36F8F9368986EF6
:100C7000704700BFE8000020B428000000ED00E04D
:100C8000202080F31188BFF36F8F11498A684FF0DD
:100C900028001044EFF3098C80E8F01F0D4F4FF04F
:100CA00000664A6A8A603E60506E0023536680F395
:100CB000118804B50648806801F056FBBDE8044081
:100CC00002F1280090E8F01F8CF3098870470000BB
:100CD000E800002004ED00E01EF0040F0CBFEFF36D
:100CE0000880EFF30980816931F8021C11F0FF01DF
:100CF0000229FFD001B501F028FB01BD38B51B4C1E
:100D000005461B4801F004FBA36AD90602D5194821
:100D100001F0FEFAA36A1A0702D5174801F0F8FAA3
:100D2000A36A9B070ED5154801F0F2FA616BA36A1E
:100D3000180607D5124801F0EBFA1DB1A36A23F09B
:100D40008003A362094CA36ADA0702D50D4801F0BB
:100D5000DFFAA36A9B0602D50B4801F0D9FAA36A11
:100D6000A36A43F0FF03A362002038BD00ED00E05A
:100D7000742A00008B2A0000BF2A0000D32A00003A
:100D8000EC2A0000032B0000232B000038B51E4C7A
:100D900005461E4801F0BCFAA36AD90402D51C48D6
:100DA00001F0B6FAA36A1A0502D51A4801F0B0FAA2
:100DB000A36A9B050ED5184801F0AAFAA16BA36A95
:100DC000180407D5154801F0A3FA1DB1A36A23F44E
:100DD0000043A3620C4CA36A590502D5104801F0E8
:100DE00097FAA36ADA0509D50E4801F091FA064A86
:100DF000936A43F47F439362002038BDA36A9B0447
:100E0000F5D50948F1E700BF00ED00E01329000027
:100E10002A290000BF2A00003C29000056290000B2
:100E20006C29000088290000232B000010B5194C04
:100E3000194801F06DFAA36A9A0102D5174801F02A
:100E400067FAA36ADB0102D5154801F061FAA36ACB
:100E5000180302D5134801F05BFA0E4CA36A59033C
:100E600002D5114801F054FAA36A9A0302D50F483B
:100E700001F04EFAA36ADB0302D50D4801F048FAEF
:100E8000044A936A6FEA03436FEA134393620020B4
:100E900010BD00BF00ED00E0532B00006C2B0000E4
:100EA000802B00009B2B0000BA2B0000E02B0000E1
:100EB000FB2B000038B5274C6368C3F30803DA1E28
:100EC0000546092A3AD8DFE802F0053335303939CA
:100ED00039393937204801F01BFAE36A9A0703D5FC
:100EE0001E4801F015FA02E0E36A5B0005D4002019
:100EF0002946BDE8384000F0D1B8194801F008FA99
:100F0000184B1B782BB10120FFF7F8FE0628EFD114
:100F100038BD154B1B781BB10120FFF737FFF5E7F4
:100F2000124B1B889BB2002BE1D0FFF77FFFEDE750
:100F30000020E9E70020F0E70D48D2E70D480E4910
:100F4000A3F110020F2BD8BF01460C4801F0E0F9C5
:100F5000CDE700BF00ED00E0CF290000E729000049
:100F6000092A000028ED00E029ED00E02AED00E06C
:100F7000292A0000A1290000B6290000602A0000EB
:100F8000024A536943F010035361704700ED00E0DB
:100F900043B2002B08DB012200F01F0002FA00F030
:100FA0005B09024A42F82300704700BF00E100E0FD
:100FB00043B2002B0DDB01225B0900F01F0002FA97
:100FC00000F02033034A42F82300BFF34F8FBFF3F2
:100FD0006F8F704700E100E043B2002BA8BF03F120
:100FE000604301F101014FEA4111AEBF03F56143D6
:100FF00000F00F00034BC9B2ACBF83F800131954C3
:10100000704700BF14ED00E02DE9F0418C188846D0
:1010100017461E4604220A9B0999054601F0D6FA96
:10102000A4F120030C4923F00703002221F0010161
:10103000C5E91322C5E91687996106995960079990
:1010400099600899D9604FF080711E60D961AB64D6
:101050006A66BDE8F08100BF25200000014910222A
:101060000A60704710ED00E0404080F3118830BF07
:10107000704700BF404080F31188DFF81CC0DCF8E7
:1010800000C01CF4006C0CBFEFF30880EFF3098084
:1010900001B5FFF70FFF01BD04ED00E038B50446D0
:1010A0000D4605281AD8DFE800F0031919131517A3
:1010B0000D4801F02DF900F099FDAA6901460B4891
:1010C00001F026F929462046BDE8384000F018B85E
:1010D0000748EEE70748ECE70748EAE70146074814
:1010E00001F016F9E7E700BF272C0000C52C00002F
:1010F000472C00006D2C0000872C0000A22C000063
:10110000052810B50CD000F077FD60B100F074FD3B
:101110000C490D4B002808BF19460C4801F0F8F89F
:10112000FFF7A2FFFCE700F077FD0028EED1084CA6
:101130000848A16801F0ECF8A068BDE8104000F094
:101140000BB800BF012D0000052D0000162D00007A
:10115000E8000020362D000038B505464FF020038A
:10116000EFF3118483F31188BFF36F8F01F00FFA4F
:101170000A4B9B68AB420BD1094B5A68C2F3080279
:1011800012B92046FFF762FD5A6842F080525A6059
:101190002046BDE8384001F0A1B900BFE8000020BA
:1011A00000ED00E001B572B60B4A106A00281EBFC0
:1011B0000021116201F060F962B6EFF30580A0F141
:1011C00010004FEAC0000549014409C99847BDE82D
:1011D0000140034800470000E800002068260000A6
:1011E000190C000001F0B5F800F004F830BFFFF76B
:1011F000FDBF00BF08B50E4B83F30988EFF31483DE
:1012000043F0020383F31488BFF36F8F094B0A4A3C
:1012100023F07F039360BFF34F8FBFF36F8F00F016
:101220007FFA00F087FAFFF705FD00F0B5FA00BF7E
:10123000700E00200000000000ED00E01FB5094B1B
:101240000193094B029304A8084B039301AB40F8A8
:10125000103D074A074B012100F076F805B05DF814
:1012600004FB00BF000000200000000000000B068F
:10127000000000200000042030B5D1E90043202BFD
:10128000896817D9B3F1004F16D8013BB3FA83F33D
:10129000C3F11F035B00072841F001010ED824F0C1
:1012A0001F02084D024342F010020B43A860EA609F
:1012B0002B6130BD0823EEE73E23ECE76FF015000D
:1012C000F7E700BF90ED00E0034B05225A60BFF343
:1012D0004F8FBFF36F8F704790ED00E0BFF35F8FCC
:1012E000014B00225A60704790ED00E013490868F6
:1012F000082810B51ED8FFF7F1FF114C49680022ED
:10130000904201F10C0105D10E4B1870FFF7DCFF84
:10131000002010BDA26051F80C3C23F01F0343F0E5
:1013200010031343E36051F8043C43F001032361CD
:101330000132E5E74FF0FF30EBE700BF5428000033
:1013400090ED00E02B010020F8B5104C0746207806
:101350000E460025B54208DA57F825104B6893B1C0
:101360005A1E134203D06FF015002070F8BD1F2BDA
:10137000F9D90B681A42F6D1C0B2FFF77DFF10F120
:10138000160FF0D001300135E4E700BF2B0100203B
:1013900070B5104B064618780D460024AC4207DBAA
:1013A00010F1160F03D00C4B002207280DDD70BD85
:1013B00056F824104B6833B1C0B2FFF75DFF10F14F
:1013C000160FF4D001300134E8E798601A6101305B
:1013D000EBE700BF2B01002090ED00E0014B18600F
:1013E000704700BF780E002038B50A4800F058F961
:1013F0000546094800F054F90622044607492846E4
:1014000001F018F820460822054901F013F80020E1
:1014100038BD00BF5B2D0000622D0000692D00006B
:10142000752D0000034B186818B1D3F85C03C3F89E
:101430005C0370472421004030B54B79012B20D14B
:101440008B79032B1DD1CC792CB1012C19D10368D8
:101450009B681B78ABB10A7912B1022A11D10E2216
:101460000B6847F61225AB426CD027D8B3F5965FD0
:1014700061D012D8B3F5167F4CD005D8B3F5967F5E
:1014800070D06FF0220052E0B3F5966F50D0B3F5F4
:10149000166FF6D14FF41D233EE0B3F5615F4CD0DB
:1014A00004D8B3F5165FECD1304B35E0B3F5964F69
:1014B00046D0B3F5E14FE4D12D4B2DE0B3F5E13F3C
:1014C00048D011D84DF6C025AB423ED004D8B3F574
:1014D000164FD6D1274B1FE0B3F5614F38D0B3F587
:1014E000963FCED1244B17E0B3F5E12F36D008D884
:1014F000B3F5613F30D0214DAB42C2D14FF0806394
:101500000AE0B3F5612F2BD01D4DAB42B9D14FF09E
:10151000805301E04FF41C331A4D2243C5F82435A3
:10152000C5F86C25836803C983E80300002030BD3B
:101530004FF49E23F0E7144BEEE74FF46C13EBE708
:10154000124BE9E74FF40003E6E74FF46503E3E7E6
:101550000F4BE1E70F4BDFE70F4BDDE70F4BDBE70F
:101560000F4BD9E74FF4A033D6E700BF0050270058
:1015700000F0750000509D0000903A0190D00300EB
:1015800040420F000020004000B0130000A04E00B9
:1015900000F0EB0000E0D70100B0AF0300705F0780
:1015A00000D0BE0E084B1A6882B052B100201860FD
:1015B0001B680193019B054BD3F818350B7002B0E3
:1015C00070474FF0FF30FAE708210040002000404C
:1015D000094B00221A6082B01A680192019A074AE8
:1015E00001201060C2F814151A68002AFCD0044BC0
:1015F00001221A6002B070471C2100400820004000
:101600000C2000404FF0A04373B52022164CC3F8C5
:101610000825002103220525C3F81427C3F80C1759
:10162000C4F81425C4F80C55104D4FF48076C5F855
:101630000865C5F82027C3F81C172823C4F8083507
:101640000723C4F810358168FFF7F6FE48B9042374
:10165000C4F80035064B18601B680193019B0123F9
:10166000236002B070BD00BF0020004000030050A6
:1016700008210040094B70B553F820400130002686
:1016800053F82050A54200D870BD236820465B68FF
:10169000984700B166600C34F4E700BFA028000052
:1016A000104B70B5104C05461E469C4204D10E4CA2
:1016B000B44209D1002412E062681AB122681268AB
:1016C000AA420CD00C34F0E763680BB90C34EFE796
:1016D00023682846196800F04FFE0028F6D12046FE
:1016E00070BD00BFF80E00208C0E002008B50B4D19
:1016F0004FF02002EFF3118382F31188BFF36F8F55
:1017000000F082FF012102280446D8BF084600F0FD
:101710008BFF2C62FFF7A8FCEAE700BFE80000207F
:101720000248034A0021121A00F060BE00000020A7
:101730003001002008B50648064A0749121A00F091
:1017400028FE064A06490748BDE8084000F021BEC9
:10175000700E00200C0F0020D02D000000000000B3
:10176000D02D00000000002008B50220FFF782FF06
:10177000074800F0CDFD0320FFF77CFF00F092FA50
:10178000FEF776FE034A137B23F00103137308BDB3
:10179000862D00007C00002080B53D4BA2B083F375
:1017A00008883C4B3C4E5A693C4D42F400725A61E9
:1017B0000024E02283F82220DC771C765C769C767D
:1017C0005A6A42F4E0225A62FFF7DAFBFFF746FC5E
:1017D00007AB21466C22184600F008FE0127B060D6
:1017E00020468DF82970FFF745FF3846FFF742FF86
:1017F00000F0F0F92A4B75624FF48062CDE9047372
:10180000CDE90244CDE90044264B2749284600F0A3
:101810002FFA6B7B23F0040213F01B0F6A7334461C
:1018200004D1AB6913B9284600F002F91F4B204ED2
:10183000059301220F23CDE9033200234FF4A07258
:101840001C4900933046CDE901331B4B00F010FAE0
:10185000737BE66023F004037373184BC4E906330B
:10186000FFF7ECFC0D48A56000F07EFD0D4B144A1F
:10187000184682F3098863B64FF0000181F311889E
:10188000BFF36F8F00210022002300F0CBFB00BFCD
:10189000700E002000ED00E0E80000207C00002039
:1018A000C62D00006917000030010020CB2D00007C
:1018B0001000002030050020ED160000000100207F
:1018C00030050020EFF305800D2809D828B1054B1D
:1018D000586880F40060C0F3C02080F001007047B9
:1018E0000120FAE700ED00E008B5FFF777F9054BB6
:1018F000054A1B681844106100211846BDE80840DD
:1019000000F092BE20010020E8000020F8B50D464E
:101910004FF02003EFF3118483F31188BFF36F8F2F
:101920000D4E0E4B4FF400410027C1FB0067002213
:101930001A6130464FF4A02200233946FEF7E0FB3F
:10194000074B1860074B1D60FFF7CEFF84F311882B
:10195000BFF36F8FF8BD00BFFFFF0400E800002059
:10196000200100201C0100204FF02003EFF3118123
:1019700083F31188BFF36F8F044B9A68D37B013BCD
:10198000D37381F31188BFF36F8F7047E800002095
:10199000094B03F12802824205D19B688B4202D198
:1019A0004B7BDB0607D1D1E900231A600A6853603C
:1019B0000023C1E900337047E800002038B50D4C22
:1019C000024604F1280000F0A2FD054600B9E568D2
:1019D000A3684AB95A7BD20606D1AA6922B9DA8924
:1019E0007F2A01D9636238BD9D4201D0FFF77CFF99
:1019F0006562F8E7E800002010B54FF02003EFF330
:101A0000118483F31188BFF36F8F084B9A68D37BDF
:101A10000133D3730120FFF7D1FF84F31188BFF3A3
:101A20006F8FBDE8104000F068BD00BFE8000020E7
:101A3000F8B54FF02003EFF3118483F31188BFF35F
:101A40006F8F164A114651F8283F8B420CD05BB17C
:101A5000D66A90F90E5093F90E70AF420BDCB34288
:101A600002D01B68002BF6D1D36A4360D36A0160B1
:101A70001860D06205E05A68C0E900325A68106008
:101A80005860437B43F0400343730020FFF796FF09
:101A900084F31188BFF36F8FF8BD00BFE80000200A
:101AA000F8B504464FF02003EFF3118683F3118855
:101AB000BFF36F8F194F07F1280501462846FFF73E
:101AC00067FFBB6AAB423A460CD05BB1F86A94F947
:101AD0000E1093F90E708F420BDC834202D01B680C
:101AE000002BF6D1D36A6360D36A25601C60D46290
:101AF00005E05968C4E9003159680C605C60637B9B
:101B0000906843F040036373031B58425841FFF74A
:101B100055FF86F31188BFF36F8FF8BDE8000020F2
:101B20001449154A8B6810B51468A34203D1BDE867
:101B30001040FFF7D9BE00241460104A1268BAB1F1
:101B4000DA897F2A14D80E4A93F90E40126894421B
:101B50000EDB0C4A126893420AD09A6942B90A69AC
:101B6000824203DC1846FFF79BFFE0E7121A0A6186
:101B700010BD00BFE8000020180100202001002057
:101B80001C010020B828000038B504464FF020039F
:101B9000EFF3118583F31188BFF36F8F437B5A06F0
:101BA00007D501460948FFF7F3FE637B23F04003A6
:101BB0006373074B9868031B58425841FFF7FEFEBA
:101BC00085F31188BFF36F8F38BD00BF100100206F
:101BD000E8000020044B002103F12802C3E90A2297
:101BE0000846FFF793BE00BFE8000020014B98684D
:101BF000704700BFE8000020EFF305800D2807D8EC
:101C000038B1044B586880F40060C0F3C0207047BE
:101C10000120704700ED00E0024B9B68187B00F04C
:101C200001007047E800002010B502464FF0200385
:101C3000EFF3118483F31188BFF36F8F437B590750
:101C400004D484F31188BFF36F8F10BD23F0040315
:101C5000437300F093FC10B11046FFF7E9FE2146F4
:101C60000248BDE8104000F02BBC00BF2C01002052
:101C700030B587B004460E9D04950D9D03950C9DCF
:101C800002950B9D01950A9D0095FFF7BDF9044B48
:101C90009B6813B9236607B030BD1B6EFAE700BF1F
:101CA000E80000202DE9F04F284E294D87B0B046BE
:101CB000B54205F130040FD3FFF756FE244C254EF4
:101CC000DFF894A04FF400490027444521D307B022
:101CD000BDE8F04FFFF790BE54F8043C059354F86C
:101CE000103C049354F8143C039354F8183C0293AA
:101CF00054F81C3C019354F8203C009354E90A2307
:101D000054E90C01FFF7B4FF54F8303CDD6425467C
:101D1000CEE7616A4B1C04D0256821B92846FFF73D
:101D200083FF3034D1E7B346BC46C9FB01BC4FF456
:101D3000A022002358466146FEF7E2F95146421CB4
:101D400005F1180000F052F8EBE700BFF80E002094
:101D5000F80E0020FFFF04001B250000034B1B684A
:101D60000BB9FEF73BBF0020704700BF24010020E5
:101D7000036840B1084A5268904204D01BB19A6887
:101D800081680A449A604268136003685A600023BD
:101D9000C0E90033704700BF840E002038B5104BF7
:101DA0001B78002B0F4B1C6814BF4FF0FF306FF0F7
:101DB00000409C420AD04CB1A568FFF7CFFF281A1B
:101DC00000280ADBA468FFF7C9FF201A064B1B692D
:101DD00013B19842A8BF184638BD0020F6E700BFEF
:101DE0002C010020840E0020E800002070B504467D
:101DF0001646C1604FF02003EFF3118583F311887D
:101E0000BFF36F8FFFF7AAFF194B1A68012EACBF03
:101E1000801901309A42A06001D05E6832B95A68D8
:101E200062605A68236014605C600BE09068A1688F
:101E3000884216DD411A91605168C4E90021516859
:101E40000C6054601A689A4206D0944204D1FFF79D
:101E5000A5FF0021FEF788FE85F31188BFF36F8F81
:101E600070BD091A9642A160D9D01268D6E700BFAA
:101E7000840E00202DE9F04B0446FFF751FE4FF091
:101E80002003EFF3118583F31188BFF36F8F214E89
:101E9000214FDFF888903460B846D9F800403268A6
:101EA0004C45D7E900BC05D024B1A368934214DDAA
:101EB0009B1AA3601BEB02004CEBE2710024C8E903
:101EC00000013460FFF76AFF2146FEF74DFE85F3FF
:101ED0001188BFF36F8FBDE8F08B1BEB03004CEB59
:101EE000E371D31A33600023C7E90001A3602046E1
:101EF000FFF73EFF85F31188BFF36F8FE3689847C4
:101F00004FF02003EFF3118583F31188BFF36F8F38
:101F1000C3E700BF2401002000000020840E002041
:101F200038B5074C074DAC4201D3002038BD04F151
:101F300014032046C4E9053300F029F81C34F2E705
:101F4000F80E0020F80E002070B5C66890F90B005E
:101F50000C254D43884206EB0504B4BF7159214658
:101F6000202492FBF4F401EB8401196002F01F00BD
:101F700070BD07B501ABFFF7E7FF019A012303FA34
:101F800000F013680343136003B05DF804FB2DE910
:101F9000F843044643680589006894F80AC05D4325
:101FA000FF222844E27200214FF00C0E8C4505DC24
:101FB00000252389AB4222DCBDE8F883D4F80C80ED
:101FC000B5FBF3F20EFB01F71F2A08EB0706C8BFAB
:101FD0001F324FEA930306F10409C8BF520903F107
:101FE0000303C6E9019923F00303D4BFE17248F863
:101FF000070001F10101C8BF00EB8200D6E762686B
:10200000E36820686A4381181E1D86509A684A60FA
:102010009A682046116099602A460021FFF7A9FFBF
:102020000135C6E708B50446084611461A46A047DA
:10203000FFF7DCFDFFF790F80020704770B504460D
:102040000D464520A04729465220A0472946234651
:102050005220BDE8704018472DE9F04F89B01C466A
:102060004FF0000A531E06460F4603934FF0FF3908
:10207000D046002505E06DB9252800F03D813946A0
:10208000B047039B13F8010F03930028F3D109B065
:10209000BDE8F08F642862D019D839280AD83128D1
:1020A00051D22D283DD030283ED0252808D13946A0
:1020B000B047DEE7582800F0A880632800F01681BA
:1020C00039462520B047039B39461878F0E7702839
:1020D00000F0918006D8692841D06C283CD068284F
:1020E000CFD0EDE775286DD017D87328E8D12568D3
:1020F00004F1040B2B461C4614F8010B002840F099
:10210000EC80B8F1030F40F000815C1BA9EB0404E4
:10211000002C00F3E6805C46ABE7782875D07A287F
:10212000DEE74FF00308ACE7B9F1000F0EDAB8F1C3
:10213000000F00F0E780A0F13009B8F1000F08BFF0
:102140004FF002089DE7B9F1000FF4DB0A2303FB0F
:102150000909A9F13009F0E70AF1010A91E7BAF19A
:10216000000F12D125680434002D05DA39462D20E0
:10217000B0476D4209F1FF39CDF8009043462A4639
:1021800039463046FEF784F973E7BAF1010FE9D01A
:10219000073424F0070303F10804D3E9002312F104
:1021A000004043F100014FF0000C4FF0FF3B8C4525
:1021B00008BF834504D239463046FFF73FFF58E752
:1021C0001546D1E7BAF1000F05D122680434CDF8E5
:1021D00000904346D4E7BAF1010FF6D0073424F05B
:1021E000070303F10804D3E90023002B08BFB2F171
:1021F000004FECD3DFE739463020B047394678202E
:10220000B0474FF008094FF00108BAF1010F27DC81
:1022100023680793002304930434002310220293BD
:1022200006939346079B0BF1FF3B4FEA8B00C0F1EF
:10223000200CA0F1200123FA00F0049B03FA0CFC0F
:1022400040EA0C0023FA01F1084310F00F0013D10B
:10225000069B13B9BBF1000F2ED14FF0300C11E0EB
:10226000073424F0070303F108041A685B68079237
:102270000493D2E7059AD5E709288CBF4FF0570C95
:102280004FF0300C394660440592B047029B0695EA
:1022900001330293BBF1000FECD1B8F1030F7FF4CF
:1022A000E8AE029BC3EB4905002D7FF7E2AE39464D
:1022B0002020B047013DF7E7531E91450593E9DB28
:1022C000B8F1010F03D139463020B047E2E7B8F149
:1022D000020FDFD139462020F7E73946B0472346C1
:1022E00009E739462020B047013C11E72068251D49
:1022F0003946B0472C46BCE6AA46A8464FF0FF39FF
:102300000125BEE64FF00108BBE65C460546B8E68F
:102310000FB407B504A951F8040B0191FEF70EF9AB
:1023200003B05DF804EB04B07047704708B50022B5
:1023300010460121FEF750FE0020FEF729FE002086
:1023400008BD70477047FEF795BE01460068FEF76E
:10235000A5BE202383F31188704708B5FEF746FF1A
:10236000BDE80840FEF758BC07B5002101A8FFF7FB
:102370000FF803B05DF804FB0138013910F8013F94
:1023800011F8012F934202D1002BF7D11A46981A67
:102390007047F0B581EA0004A50703460BD0013B66
:1023A0000A4491421DD1F0BD002AFCD011F8014B26
:1023B00003F8014B013A9C07F6D11D1F0C468F18FC
:1023C0003E1B032E08D894086FF0030505FB04227A
:1023D000A40023442144E2E754F8046B45F8046F59
:1023E000EEE711F8014B03F8014FDAE7F0B5C9B297
:1023F00003469C070FD141EA012444EA04441D46E8
:102400009F187E1B032E0CD8940803EB84041344FE
:102410009C4209D1F0BD002AFCD003F8011B013A0F
:10242000E7E745F8044BECE704F8011BF0E74FF051
:10243000FF307047F8B505460C4601EB42066B6865
:1024400022781F68002101232846B84763786A680C
:10245000B3FA83F3576814F8022B5B09002128466E
:10246000B847B442EBD1F8BD82680B4692E803004E
:1024700083E8030000207047FFF764BF437BDB065F
:1024800003BF8069B0FA80F040090020704738B57A
:1024900004464FF02003EFF3118583F31188BFF357
:1024A0006F8F01468068FFF773FA637B23F00203A6
:1024B000637385F31188BFF36F8F0023A36038BD6A
:1024C00008B5FFF7FFF920B10846BDE80840FEF760
:1024D000BDBB81F31188BFF36F8F08BD08B50246FD
:1024E000FFF7F0F920B11046BDE80840FEF7AEBB9B
:1024F00082F31188BFF36F8F08BD4FF02003EFF315
:10250000118083F31188BFF36F8FFFF7E7BF036874
:10251000984214BF18460020704750F8103C70B520
:102520000446A0F11805CBB14FF02003EFF311865C
:1025300083F31188BFF36F8F294650F8100CFFF713
:1025400027FA14F80B3C23F0020304F80B3C86F343
:102550001188BFF36F8F002344F8103C14F80B3C34
:1025600023F0040304F80B3C2846FFF787FF20B153
:102570002846BDE87040FFF75BBA70BD437BDB06C1
:1025800003BF8069B0FA80F0400900207047036DF6
:1025900010B5044603B198472046FFF7EFFF38B166
:1025A0002046FFF7F1FA637B43F00803637310BD25
:1025B000637B9B0702D52046FFF769FFA369002BC9
:1025C000F1D004F1180000F009F8ECE703730023E0
:1025D00042738173C373C0E90633704710B54FF07F
:1025E0002002EFF3118482F31188BFF36F8F036829
:1025F0003BB1FFF7BDFB002084F31188BFF36F8F61
:1026000010BD6FF01500F7E710B54FF02003EFF3A2
:10261000118483F31188BFF36F8FFFF7BFFB84F33F
:102620001188BFF36F8F10BD70B504460E464FF092
:102630002003EFF3118583F31188BFF36F8FFFF74A
:10264000ADFBA04205DD012803DD31462046FEF743
:0E2650008BFA85F31188BFF36F8F70BD704752
:02265E00FFFF7C
:0826600040DBFF7F01000000D8
:1026680000000000A9090000000000004723000046
:10267800000000004723000000000000472300007E
:10268800000000004723000000000000472300006E
:10269800000000004723000000000000472300005E
:1026A800000000004723000000000000472300004E
:1026B800000000004723000000000000472300003E
:1026C800000000004723000000000000472300002E
:1026D800000000004723000000000000472300001E
:1026E8000000000047230000000000008D0A0000E1
:1026F80000000000472300000000000047230000FE
:1027080000000000472300000000000047230000ED
:1027180000000000472300000000000047230000DD
:1027280000000000472300000000000047230000CD
:1027380000000000472300000000000047230000BD
:1027480000000000472300000000000047230000AD
:10275800000000004723000000000000472300009D
:10276800000000004723000000000000472300008D
:10277800000000004723000000000000472300007D
:10278800000000004723000000000000472300006D
:10279800000000004723000000000000472300005D
:1027A800000000004723000000000000472300004D
:1027B800000000004723000000000000472300003D
:1027C800000000004723000000000000472300002D
:1027D800000000004723000000000000472300001D
:1027E800BE2A00005D05000000000000BE2A0000AF
:1027F800A507000000000000F52800002D230000B8
:1028080000000000FF2800002D2300000000000049
:1028180009290000D90A000000000000BE2A0000B3
:10282800ED12000000000000BE2A0000E9130000BD
:1028380000000000EE28000005160000852D0000AD
:0C284800BE2A0000211F0000000000005C
:10285400020000005C28000000000000DF280000E7
:102864002600020700000020E728000022000B11C8
:10287400F908000000000000000000003508000016
:10288400C107000000000000A5150000D1150000DC
:102894002514000039140000692400008C0E002067
:1028A400E00E0020EC0E0020F80E0020F80E0020B0
:1028B400F5FFFFFF100000206E72663532383430A9
:1028C4005F70636131303039300048656C6C6F2063
:1028D400576F726C64212025730A00464C4153489B
:1028E4005F30005352414D5F3000554152545F30C8
:1028F40000434C4F434B5F33324B00434C4F434BED
:102904005F31364D007379735F636C6F636B002ABC
:102914002A2A2A2A20425553204641554C54202A1B
:102924002A2A2A2A0A002020537461636B696E677D
:10293400206572726F720A00202050726563697399
:1029440065206461746120627573206572726F72B0
:102954000A00202042464152204164647265737328
:102964003A20307825780A002020496D707265631A
:102974006973652064617461206275732065727285
:102984006F720A002020496E737472756374696FE4
:102994006E20627573206572726F720A00526573DD
:1029A400657276656420457863657074696F6E201E
:1029B400280053707572696F757320696E7465723F
:1029C40072757074202849525120002A2A2A2A2A12
:1029D4002048415244204641554C54202A2A2A2A50
:1029E4002A0A002020427573206661756C74206F7A
:1029F4006E20766563746F72207461626C652072F8
:102A04006561640A0020204661756C7420657363F7
:102A1400616C6174696F6E20287365652062656CF2
:102A24006F77290A002A2A2A2A2A204465627567B0
:102A3400206D6F6E69746F72206578636570746958
:102A44006F6E20286E6F7420696D706C656D656E95
:102A540074656429202A2A2A2A2A0A002A2A2A2A68
:102A64002A20257320256429202A2A2A2A2A0A00B2
:102A74002A2A2A2A2A204D5055204641554C5420B2
:102A84002A2A2A2A2A0A002020537461636B696E59
:102A940067206572726F722028636F6E7465787434
:102AA4002061726561206D69676874206265206EBB
:102AB4006F742076616C6964290A002020556E7356
:102AC4007461636B696E67206572726F720A0020AD
:102AD4002044617461204163636573732056696F98
:102AE4006C6174696F6E0A0020204D4D464152207E
:102AF400416464726573733A20307825780A002043
:102B040020496E737472756374696F6E20416363D8
:102B14006573732056696F6C6174696F6E0A002067
:102B240020466C6F6174696E672D706F696E7420D6
:102B34006C617A7920737461746520707265736551
:102B440072766174696F6E206572726F720A002A00
:102B54002A2A2A2A205553414745204641554C5498
:102B6400202A2A2A2A2A0A002020446976697369BD
:102B74006F6E206279207A65726F0A002020556E8C
:102B8400616C69676E6564206D656D6F7279206133
:102B940063636573730A0020204E6F20636F707245
:102BA4006F636573736F7220696E73747275637487
:102BB400696F6E730A002020496C6C6567616C2034
:102BC4006C6F6164206F66204558435F52455455CD
:102BD400524E20696E746F2050430A002020496CC5
:102BE4006C6567616C20757365206F662074686519
:102BF40020455053520A002020417474656D70744E
:102C040020746F206578656375746520756E6465DE
:102C140066696E656420696E737472756374696F36
:102C24006E0A002A2A2A2A2A20486172647761726D
:102C34006520657863657074696F6E202A2A2A2A74
:102C44002A0A002A2A2A2A204B65726E656C2041C2
:102C54006C6C6F636174696F6E204661696C757228
:102C64006521202A2A2A2A0A002A2A2A2A2A204BCB
:102C740065726E656C204F4F505321202A2A2A2AF0
:102C84002A0A002A2A2A2A2A204B65726E656C2099
:102C940050616E696321202A2A2A2A2A0A002A2AD4
:102CA4002A2A20556E6B6E6F776E20466174616CB4
:102CB400204572726F7220256421202A2A2A2A0A4A
:102CC4000043757272656E74207468726561642065
:102CD4004944203D2025700A4661756C74696E670D
:102CE40020696E737472756374696F6E20616464B5
:102CF40072657373203D20307825780A0049535259
:102D040000657373656E7469616C207468726561C3
:102D14006400466174616C206661756C7420696E30
:102D240020257321205370696E6E696E672E2E2ED6
:102D34000A00466174616C206661756C7420696E6A
:102D440020746872656164202570212041626F726D
:102D540074696E672E0A004750494F5F3000475030
:102D6400494F5F31000D0118010C0106011A0108D9
:102D7400010A010E010C010501070101010301090A
:102D840001012A2A2A2A2A20426F6F74696E672059
:102D94005A6570687972204F532076312E31332E64
:102DA40039392D6E6373312D353536312D676465B0
:102DB40036396432646639303866202A2A2A2A2A47
:0C2DC4000A006D61696E0069646C6500B6
:102DD000392000000090D0032F24000000C2010021
:0C2DE00000010300840E0020840E00207F
:102DEC00E827000000000000000000004828000058
:102DFC00000000000000000024280000000000007B
:102E0C0000000000002800007428000000000000F2
:102E1C000C28000080280000000000003C28000066
:102E2C008C2800007C0E0020F4270000000000001D
:102E3C000000000018280000000000000000000046
:0C2E4C0030280000000000000000000022
:102E5800F80E0020F80E002000000000000000001E
:042E68000F00000057
:04000003000011E503
:00000001FF
